:020000000F28C7
:10000800FE00030EF1000408F2000A08F300831250
:100018007F08F400642889288B010730831299002F
:10002800703083169F0004309100093083129F00BE
:10003800F9308316920005308312920093010C3038
:1000480095000430831685008312850103308316DA
:100058008700033083128700843083168100F601FD
:100068007D30F5007508F800F7010630831281002D
:100078008B168B17F930F5000000F50B4028442843
:10008800000083129F149F1847281E08F500750862
:10009800F60007307602031855280730F500750872
:1000A800F60087185F2807185E28FF30F5007508E6
:1000B800F6005F28F6017603FF3AFF3E93003E28DC
:1000C8000B1D7E280B11063081000130F802F8085C
:1000D800031D76287D30F0007008F8000430F00029
:1000E8007008F700770803197D280130F702071612
:1000F8007E2807127408FF0073088A0072088400BB
:10010800710E8300FE0E7E0E0900F601F7018301D1
:020118001028AD
:02400E00E1F3DC
:00000001FF
